:020000040000FA
:0A0000000000000049EF01F05FD19D
:0800180096D19EA8FED7AD6E43
:1000200012000C6A0B6EFF0E0B260C2200D0D8A01B
:100030001200030E0A6EE60E02D8F5D70A6AFE0F0A
:10004000096EE86A0A5AD8A012000000090600D01A
:10005000F8D71450105C196E11E2196C105014C0CE
:1000600010F0146E115015C011F0156E125016C01C
:1000700012F0166E135017C013F0176E1A0E196097
:1000800074D0145272E0186A11501C6E15181B6E51
:10009000118E158E080E195E08E317C018F016C0F1
:1000A00017F015C016F0156AF5D7192607E0D89095
:1000B0001532163217321832192EF9D71BAE33D03B
:1000C0001750135E1650125A1550115A07E2D88075
:1000D000000E135612561156800E1C1A186C04E0AE
:1000E0001306000E125A115A040E196E11660DD025
:1000F00012C011F013C012F018C013F0186A080EE5
:10010000105E29E3192EF2D726D011BE08D0D89060
:100110001836133612361136102EF7D71CD018AEFB
:1001200022D0186A0FD017501326165012221550DD
:10013000112206E31132123213321832104A0DD056
:1001400018AE11D0133E0FD0123E0DD0113E0BD081
:10015000D8801390EFD7106A02D01A821068136A01
:10016000126A800E116E1CAE119E1350120010C048
:100170001CF0115013C011F0136E13361C321332E1
:100180001A6A13361C3602E31A841A7E06E11A80B4
:100190001C6A136A126A116A0BD01C2803E0D8800B
:1001A000133206D0D890133202E11A8201D01A8697
:1001B0001AB604D01AA20FD01AB407D07F0E136E4D
:1001C000FF0E126E116E106E23D0800E136E01D0D2
:1001D000136A000EF6D71AB0FBD7106A9F0E1C6088
:1001E000EBD77E0E1C64F4D79E0E1C5C07E0D89003
:1001F00013321232113210321C2AF6D71AA408D048
:10020000D880000E105611561256135613AEE0D772
:1002100010501200126A136A1B9E0AD01B9E13AE66
:1002200007D0D880000E10561156125613561B8E4A
:10023000960E1C6E135209E0080E1C2611C010F019
:1002400012C011F013C012F011D012520FE1080EBB
:100250001C5E115007E1080E1C5E105002E11350A5
:1002600010D0106A126E10C011F0106A12BE06D0C3
:10027000D8901036113612361C06F8D71BAE129ED7
:100280001C5010C013F0106E125011C012F0116EFD
:100290001200400E1A6E006AB8964F0EAF6EB06A2A
:1002A000240EAC6E900EAB6E00010F0EC16E070EE9
:1002B000B46EC69AC00E926EE00E936EC00E946E2F
:1002C000956AE80E966E52D0F2A409D0F2941F4AB5
:1002D000202AD6CF1DF0D7CF1EF0817A11009EAA1A
:1002E00019D0060EAB1412E1E2CF33F0E1CF32F0B9
:1002F000342A10EE48F03450E126000EE222AECF50
:10030000E7FF33C0E2FF32C0E1FF1100AE50AE5054
:10031000AB98AB881100346A356A9D8A9F8AF28E49
:10032000F28C12009D9A00EE48F0010EF46EF36A12
:10033000F306000EF45AEE6AF450F310F9E1346A51
:10034000356A9D8A1200F29EE0CFCBF2D8CFCCF274
:10035000E8CFCDF2F28E0001A192F29ECBC2E0FF77
:10036000CCC2D8FFCDC2E8FFF28E1000939A8A9AD1
:100370000A0E57DE94928B9295948C9494988B9855
:1003800095988C98959C8C9C93908A9093948A9441
:1003900093988A9896928D92929A899A9296899633
:1003A0009292899294908B9095968C96949A8B9A2F
:1003B000959A8C9A959E8C9E93928A9293968A9601
:1003C00096948D9496908D90929889989290899019
:1003D0009294899400EE3CF00C0EEE68E82EFDD766
:1003E0009ADFA0DFCD6AF294F28A870ED56EB16AE9
:1003F000A192A082D08EA292B10EB16EE1D943EC4F
:1004000004F0B60E0ADE780E08DE400E06DED6CF09
:100410001DF0D7CF1EF067D9C9C221F0B70E215CFD
:1004200006E3FE0E215C01E301D0236A07D121AE71
:1004300021D0236A860E215C05E121C023F02468C7
:10044000256817D0960E215C05E121C023F02668AF
:1004500027680FD0A60E215C05E121C023F0366885
:10046000376807D0B60E215C04E121C023F028686C
:100470002968DDD0235202E1E1D0D9D0860E235C79
:1004800035E1242803E121C024F02ED021C025F03D
:1004900024503A5C26E13A6A550E1D24026E550E30
:1004A0001E20036E000E1F20046E000E2020056E1D
:1004B00002C03CF003C03DF004C03EF005C03FF078
:1004C00024C03BF08992899A8D928A988A908C9860
:1004D0008C9443684268416840684768466845684C
:1004E00044682468010148810001A1D0960E235C74
:1004F000D8A492D0262803E121C026F08CD021C0B8
:1005000027F0350E265CD8A084D06B0E265CD8B0C0
:1005100080D03F683E683D683C6802EE49F0265056
:10052000EB50396E02EE49F03B50EB50226E39B081
:1005300005D08994898022B0898604D089848990E5
:1005400022A0898239B205D089988D8022B28D820D
:1005500004D089888D9022A2898A39B405D08D94DF
:100560008A8622B48A8404D08D848A9622A48A88BA
:1005700039B605D08A928C8E22B68C8C04D08A82B1
:100580008C9E22A68A8039B805D08C9A8B8A22B894
:100590008B8804D08C8A8B9A22A88C8839BA05D093
:1005A0008C968B8022BA8B8204D08C868B9022AA68
:1005B0008C8426C03AF085C127F027501D24026E96
:1005C000000E1E20036E000E1F20046E000E202061
:1005D000056E02C040F003C041F004C042F005C007
:1005E00043F07BC127F027501D24026E000E1E2011
:1005F000036E000E1F20046E000E2020056E02C048
:1006000044F003C045F004C046F005C047F00101C6
:100610004881000126680BD0B60E235C08E128282B
:1006200003E121C028F003D021C029F0BAD801018C
:100630004831000103E377D8CAC230F0030E305CC2
:10064000D8B049D02C501D5C2D501E582E501F582C
:100650002F50205832E32F8E305212E18994899026
:1006600089988D908D948A968A928C9E8C9A8B9A7A
:100670008C968B903F683E683D683C683B6A1BD017
:10068000010E305C0BE18992899A8A988A908C9845
:100690008C9443684268416840680DD0020E305C1B
:1006A0000AE189968D928A948C9C8B988B924768EC
:1006B00046684568446801014881000120AE0AD0BF
:1006C000206A1F6A1E6A1D6A00EE3CF00C0EEE687E
:1006D000E82EFDD706D020AE04D0206A1F6A1E6A1D
:1006E0001D6A95D6FFD73450355C16E0352AEACF1F
:1006F0000AF0E9CF09F000EE48F03550E926000E87
:10070000EA22EF500201C96F0AC0EAFF09C0E9FFFF
:10071000D8801200000105D0E8680201C96FD8A096
:100720001200000112000201CA692F8E226A000124
:10073000D8902234E96EEA6AEA36E936EA363C0EA7
:10074000E926000EEA22EFCF02F0ECCF03F0ECCF67
:1007500004F0ECCF05F02C50025C2D5003582E50C5
:1007600004582F50055815E2D8902234E96EEA6AF1
:10077000EA36E936EA363C0EE926000EEA22EFCFE9
:100780002CF0ECCF2DF0ECCF2EF0ECCF2FF022C0E0
:10079000CAF2222A030E225CCAE301014891000139
:1007A0001200420E285C06E1295202E1E3D801D092
:1007B00003D904D07B0E285C01E1FED82868120022
:1007C00001014C6B340E4B6F020E226E0001800E45
:1007D000225C36E22204086E01EE49F0D89008341B
:1007E000E926000EEA22EECF06F0EFCF07F006C0B2
:1007F00010F007C011F00AEC01F010C014F011C0A5
:1008000015F012C016F013C017F0330E136E126EEF
:10081000030E116E840E106E29EC00F0B7EC00F0A0
:10082000026E11C003F001EE49F0D8902234E9269F
:10083000000EEA2202C0EEFF03C0EFFF222AC6E349
:10084000010E226E800E225C1DE201EE49F0D8906E
:100850002234E926000EEA22EECF06F0EFCF07F0B1
:10086000D8900730036E0630026E01EE49F0D89042
:100870002234E926000EEA2202C0EEFF03C0EFFF99
:10088000222AE0E31200226A360E225C08E2F36AB2
:1008900002EE49F02250F3CFEBFF222AF5E30201EA
:1008A0003F0E7E6F7F6F806F816F826F836F3E0E12
:1008B000846F3D0E856F3C0E866F280E876F350E58
:1008C000886F300E896F280E8A6F200E8B6F100E86
:1008D0008C6F300E8D6F100E8E6F8F6F906F916FCB
:1008E0003F0E926F936F946F956F966F3E0E976F5A
:1008F0003D0E986F3B0E996F380E9A6F340E9B6FBA
:10090000300E9C6F280E9D6F200E9E6F100E9F6FF5
:100910001F0EA06F1D0EA16FA26F180EA36F350ED4
:10092000A46F370EA56FA66F270EA76F280EA86FAE
:10093000A96F360EAA6F240EAB6F1F0EAC6F1D0E83
:10094000AD6FAE6F180EAF6F350EB06F370EB16F63
:10095000B26F200EB36F6B0E226E0001800E225C10
:1009600008E2F36A02EE49F02250F3CFEBFF222AAD
:10097000F4E3120000EE3CF00C0EEE68E82EFDD71A
:100980008C948B928C988B988C9C8A908A948A9861
:100990008D92899A899689928C968B908C9A8B9A53
:1009A0008C9E8A928A968D948D908998899089944C
:1009B000010148810001120000EE3CF00C0EEE68CF
:1009C000E82EFDD78C948B928C988B988C9C8A9077
:1009D0008A948A988D92899A899689928C968B901E
:1009E0008C9A8B9A8C9E8A928A968D948D908998F7
:0C09F000899089940101488100011200E7
:020000040030CA
:0300010006160ED2
:020005008580F4
:060008000FC00FE00F40E5
:00000001FF
